:020000040000FA
:10000000B6EF12F01200FFFFFFFFFFFFFFFFFFFF41
:10001000FFFFFFFFFFFFFFFFFAEF10F01200FFFFEF
:10080000B6EF12F01200FFFF1200FFFFFFFFFFFF25
:10081000FFFFFFFFFFFFFFFF1200FFFFFFFFFFFFD4
:10082000FFFFFFFFFFFFFFFFFFFF02009C2500000F
:1008300018010000010000008E250000E500000006
:100840000E000000F00E8C1695169388938A938CF8
:10085000938E8150200B01E0010E0001606F8150EA
:10086000100B01E0010E616F8150800B01E0010E61
:10087000626F8150400B01E0010E636F55EC0EF08A
:100880009280010EC26E3C0EC06EC08E07DA00016F
:10089000666B970ED56E1200D9CFE6FFE1CFD9FF78
:1008A000D950FB0FE96EFF0EDA20EA6E720E096E68
:1008B000010E0A6E0B6A0C6AEECF04F0EECF05F063
:1008C000EECF06F0EFCF07F01AEC12F003C0EDFF09
:1008D00002C0EDFF01C0EDFF00C0EFFFD950FB0FDC
:1008E000E96EFF0EDA20EA6EEF06EECF10F0000E92
:1008F000EF5AEECF11F0EF5AEECF12F0EF5AEFCFE2
:1009000013F0105011101210131001E0E7D7E55248
:10091000E7CFD9FF120080CFEAF00001E551EA17D6
:1009200081CFEBF0E651EB1782CFECF0E751EC17FB
:1009300083CFEDF0E851ED1784CFEEF0E951EE17DB
:10094000120080CFEAF00001E51DEA1381CFEBF041
:10095000E61DEB1382CFECF0E71DEC1383CFEDF037
:10096000E81DED1384CFEEF0E91DEE131200000137
:10097000EF6B0F0EC16E92689468936895689668E5
:10098000939481840A0EE66EE66AE66AE66A84DF7C
:10099000E552E552E552E552D4DFFF0E0001EA5D73
:1009A0000CE1FF0EEB5D09E1FF0EEC5D06E1FF0ED1
:1009B000ED5D03E1FF0EEE5D03E0010EEF6F3BD155
:1009C0000F0EC16E926894689368956896689394C8
:1009D00081940A0EE66EE66AE66AE66A5DDFE55233
:1009E000E552E552E55297DF0001EA5108E1EB518B
:1009F00006E1EC5104E1ED5102E1EE5103E0020E9B
:100A0000EF6F19D10F0EC16E926894689368956864
:100A1000966893948184F06B080EE76EF019E8AE47
:100A200002D0E73402D0E750F05D49E2010EF0C099
:100A3000E7FFE75204E0E846FE0BE706FCE10001B1
:100A4000E71501E13AD0010EF0C0E7FFE75204E0FC
:100A5000E846FE0BE706FCE1E81C946E010EF0C0D0
:100A6000E7FFE75204E0E846FE0BE706FCE1E81C7E
:100A7000826E0A0EE66EE66AE66AE66A0DDFE55207
:100A8000E552E552E5525DDF010EF0C0E7FFE752A7
:100A900004E0E846FE0BE706FCE1E81C0001EC5D23
:100AA00002E0030EEF6FFF0EED5D02E0030EEF6F4D
:100AB000FF0EEE5D02E0030EEF6FF02BADD70F0ED1
:100AC000C16E9268946893689568966893948184DF
:100AD000F06B080EE76EF019E8AE02D0E73402D0F2
:100AE000E750F05D4AE2010EF0C0E7FFE75204E094
:100AF000E846FE0BE706FCE10001E81501E13BD00A
:100B0000010EF0C0E7FFE75204E0E846FE0BE706FF
:100B1000FCE1E81C956E010EF0C0E7FFE75204E02F
:100B2000E846FE0BE706FCE1E81C836E0A0EE66E63
:100B3000E66AE66AE66AB0DEE552E552E552E5525B
:100B400000DFFF0E0001EC5D02E0030EEF6F010E0F
:100B5000F0C0E7FFE75204E0E846FE0BE706FCE1E1
:100B6000E81C0001ED5D02E0030EEF6FFF0EEE5D8D
:100B700002E0030EEF6FF02BACD70F0EC16E926840
:100B8000946893689568966893948184F06B080ED6
:100B9000E76EF019E8AE02D0E73402D0E750F05D1E
:100BA0004AE2010EF0C0E7FFE75204E0E846FE0B20
:100BB000E706FCE10001E91501E13BD0010EF0C0C0
:100BC000E7FFE75204E0E846FE0BE706FCE1E81C1D
:100BD000966E010EF0C0E7FFE75204E0E846FE0B18
:100BE000E706FCE1E81C846E0A0EE66EE66AE66A39
:100BF000E66A52DEE552E552E552E552A2DEFF0E0C
:100C00000001EC5D02E0030EEF6FFF0EED5D02E010
:100C1000030EEF6F010EF0C0E7FFE75204E0E84675
:100C2000FE0BE706FCE1E81C0001EE5D02E0030EAE
:100C3000EF6FF02BACD7120021D9060E0101125D27
:100C400003E36D50020B01E028D031D800016605A6
:100C500024E1F2A422D0F294480ED76EE50ED66EAF
:100C600068EC0EF0000919E00001A751E96EEA6A8C
:100C7000D890E936EA36A90EE926000EEA22F3C03A
:100C8000EEFFF4C0EDFF1E0EA85D01E2A82B1D0EC5
:100C9000A75D02E1A76B01D0A72B12000001A76B93
:100CA000A86B1200C282C2B2FED700D01200D9CF08
:100CB000E6FFE1CFD9FFE652400EE66E670EE66E24
:100CC000000EE66E2FEC10F0E552E552E5520009F9
:100CD00001E1CFD00001646B00016751FF0A01E11F
:100CE000B4D0C80A01E1A8D0010A6DE0030A63E0AC
:100CF000010A55E0070A4CE0010A2EE0030A0CE065
:100D0000310A01E0A4D00001696B0001010E6A6F95
:100D10000001040E646F9CD00001010E646F00019D
:100D2000685103E18C948C9616D00001680503E1AC
:100D30008C948C8610D0020E0001685D03E18C84D7
:100D40008C9609D0030E0001685D03E18C848C86CB
:100D500002D00001646B7CD0030E0001685D0AE1E3
:100D600000016951E8B08C84E8A08C940001010E68
:100D7000646F0DD0040E0001685D09E10001695146
:100D8000E8B08C86E8A08C960001010E646F60D0FC
:100D90000001666B83DF0001010E646F59D068ECBF
:100DA0000EF0000907E0F3C068F0F4C069F000013C
:100DB000030E646F4DD00001010E666F6FDF0001FE
:100DC000010E646F45D00001A851E824020F000114
:100DD000646F0001A851E8240001686FA8C0DFFF1C
:100DE000DF50000827E20001A75104E100011D0EB9
:100DF000A76F02D00001A7070001A751E96EEA6AB8
:100E0000D890E936EA36A90EE926000EEA22EECF9E
:100E100010F0EFCF11F0EA6ADF34FE0BEA36E96E2C
:100E2000670EE926000EEA2210C0EEFF11C0EDFFAA
:100E3000DF06D6D733DF0CD035DFC3CF68F0C4CFA1
:100E400069F00001030E646F03D0FF0001D000D0F1
:100E5000000164510EE004010CBF0BD064C0E6FF3A
:100E6000670EE66E000EE66EF5EC0FF0E552E55209
:100E7000E552E552E552E7CFD9FF12000001F151EA
:100E8000F21104E1100EF16F270EF26FF107000E60
:100E9000F25B6DA20BD0F151F21107E18C708C5016
:100EA000010B02E08C8201D08C9230D001011251F2
:100EB00004E18C908C92B0D829D0120503E18C808B
:100EC0008C8224D0020E125D03E18C808C921ED0A5
:100ED000030E125D03E18C908C8218D0050E125D1A
:100EE00007E10001F151F21102E18C708C920ED0F9
:100EF000060E125D0BE10001F151F21107E18C7059
:100F00008C50010B02E08C9201D08C821200815037
:100F1000200B01E0010E0001605D09E08150200B13
:100F200001E0010E606F81BA02D0010E02D0000E06
:100F300000D012008150100B01E0010E0001615D34
:100F400009E08150100B01E0010E616F81B802D001
:100F5000010E02D0000E00D012008150800B01E083
:100F6000010E0001625D09E08150800B01E0010E7D
:100F7000626F81BE02D0010E02D0000E00D01200BE
:100F80008150400B01E0010E0001635D09E08150DA
:100F9000400B01E0010E636F81BC02D0010E02D054
:100FA000000E00D01200D9CFE6FFE1CFD9FFACA2EE
:100FB000FED7FE0EDB50AD6EE552E7CFD9FF120033
:100FC000D9CFE6FFE1CFD9FFE652DF6ADF6ADF5013
:100FD000E76EFD0EDBCFE9FFFE0EDBCFEAFFE75049
:100FE000E926000EEA22EF5012E0DF50E76EFD0E18
:100FF000DBCFE9FFFE0EDBCFEAFFE750E926000E6C
:10100000EA22EF50E66ECFDFE552DF2AE0D7E55265
:10101000E552E7CFD9FF1200D9CFE6FFE1CFD9FFE4
:10102000E65288DF000901E15CD38C8070DF0009A3
:1010300001E1FCD78C908C827DDF000901E1FCD7B7
:101040008C928C848ADF000901E1FCD78C948C8619
:1010500097DF000901E1FCD78C96C66A948E949CB8
:10106000710EAF6E020EB06E240EAC6E900EAB6EB3
:10107000080EB86EAE50DF6EAE50DF6E0A0EE66E32
:1010800092DFE5520D0EE66E8EDFE552540EE66EEF
:101090008ADFE552650EE66E86DFE552730EE66E78
:1010A00082DFE552740EE66E7EDFE552200EE66EBC
:1010B0007ADFE552520EE66E76DFE552530EE66EAB
:1010C00072DFE552320EE66E6EDFE552330EE66EEB
:1010D0006ADFE552320EE66E66DFE552200EE66EFE
:1010E00062DFE552540EE66E5EDFE552580EE66EA4
:1010F0005ADFE552200EE66E56DFE552700EE66EC0
:1011000052DFE552720EE66E4EDFE552650EE66E78
:101110004ADFE552730EE66E46DFE552730EE66E69
:1011200042DFE552200EE66E3EDFE552420EE66EED
:101130003ADFE552330EE66E36DFE552200EE66EFC
:1011400032DFE5520ADF000901E1FCD70A0EE66E44
:101150002ADFE5520D0EE66E26DFE552540EE66EEE
:1011600022DFE552580EE66E1EDFE552200EE66ED7
:101170001ADFE552540EE66E16DFE552650EE66E96
:1011800012DFE552730EE66E0EDFE552740EE66E68
:101190000ADFE552200EE66E06DFE5524F0EE66EE0
:1011A00002DFE5524B0EE66EFEDEE552210EE66EE4
:1011B000FADEE552200EE66EF6DEE552540EE66EDD
:1011C000F2DEE552650EE66EEEDEE552730EE66E79
:1011D000EADEE552740EE66EE6DEE552200EE66EBD
:1011E000E2DEE552520EE66EDEDEE552530EE66EAC
:1011F000DADEE5522D0EE66ED6DEE552320EE66EF2
:10120000D2DEE552330EE66ECEDEE552320EE66EEB
:10121000CADEE552200EE66EC6DEE552520EE66EDE
:10122000C2DEE552580EE66EBEDEE552200EE66ED8
:10123000BADEE552500EE66EB6DEE552720EE66E8E
:10124000B2DEE552650EE66EAEDEE552730EE66E78
:10125000AADEE552730EE66EA6DEE552200EE66EBD
:10126000A2DEE552220EE66E9EDEE552520EE66EDC
:101270009ADEE552220EE66E96DEE552200EE66E0E
:1012800092DEE5529EAAFED7520EAE5C2CE1200EF5
:10129000E66E89DEE552520EE66E85DEE552580EA8
:1012A000E66E81DEE552200EE66E7DDEE552540EDE
:1012B000E66E79DEE552650EE66E75DEE552730E7A
:1012C000E66E71DEE552740EE66E6DDEE552200EBE
:1012D000E66E69DEE5524F0EE66E65DEE5524B0EB8
:1012E000E66E61DEE5520A0EE66E5DDEE5520D0E3B
:1012F000E66E59DEE552500EE66E55DEE552750E8D
:10130000E66E51DEE552740EE66E4DDEE552200EBD
:10131000E66E49DEE552650EE66E45DEE552780E74
:10132000E66E41DEE552740EE66E3DDEE552650E78
:10133000E66E39DEE5526E0EE66E35DEE552730E70
:10134000E66E31DEE552690EE66E2DDEE5526F0E79
:10135000E66E29DEE5526E0EE66E25DEE552200EC3
:10136000E66E21DEE552500EE66E1DDEE552720E8F
:10137000E66E19DEE552650EE66E15DEE552730E79
:10138000E66E11DEE552730EE66E0DDEE552200EBE
:10139000E66E09DEE552220EE66E05DEE552540EDB
:1013A000E66E01DEE552220EE66EFDDDE552200E10
:1013B000E66EF9DDE5529EAAFED7540EAE5C01E062
:1013C00005D1B7EC04F0C66A948E949C710EAF6E92
:1013D000020EB06E240EAC6E900EAB6E080EB86EA0
:1013E000AE50DF6EAE50DF6E0001EF5129E10A0E04
:1013F000E66ED9DDE5520D0EE66ED5DDE552540EF2
:10140000E66ED1DDE552650EE66ECDDDE552730E7A
:10141000E66EC9DDE552740EE66EC5DDE552200EBE
:10142000E66EC1DDE5524F0EE66EBDDDE5524B0EB8
:10143000E66EB9DDE552210EE66EB5DDE552C6D0A9
:10144000EF0541E10A0EE66EAEDDE5520D0EE66EE9
:10145000AADDE552500EE66EA6DDE552690EE66E97
:10146000A2DDE5526E0EE66E9EDDE552200EE66EC2
:101470009ADDE552740EE66E96DDE5526F0EE66E6D
:1014800092DDE552200EE66E8EDDE552470EE66EE9
:101490008ADDE5524E0EE66E86DDE552440EE66EBE
:1014A00082DDE552210EE66E7EDDE552210EE66E0E
:1014B0007ADDE552210EE66E76DDE552210EE66E0E
:1014C00072DDE55283D0020EEF5D41E10A0EE66E59
:1014D0006ADDE5520D0EE66E66DDE552500EE66EF3
:1014E00062DDE552690EE66E5EDDE5526E0EE66E79
:1014F0005ADDE552200EE66E56DDE552740EE66EBC
:1015000052DDE5526F0EE66E4EDDE552200EE66EC0
:101510004ADDE552560EE66E46DDE552430EE66EB6
:1015200042DDE552430EE66E3EDDE552210EE66EEB
:101530003ADDE552210EE66E36DDE552210EE66E0D
:1015400032DDE552210EE66E2EDDE5523FD0030E70
:10155000EF5D3CE10A0EE66E26DDE5520D0EE66E0D
:1015600022DDE552500EE66E1EDDE552690EE66E96
:101570001ADDE5526E0EE66E16DDE552200EE66EC1
:1015800012DDE552730EE66E0EDDE552680EE66E74
:101590000ADDE5526F0EE66E06DDE552720EE66E6E
:1015A00002DDE552740EE66EFEDCE552210EE66EBB
:1015B000FADCE552210EE66EF6DCE552210EE66E0F
:1015C000F2DCE552210EE66EEEDCE552C66A948E40
:1015D000949C710EAF6E020EB06E240EAC6E900E27
:1015E000AB6E080EB86EAE50DF6EAE50DF6E0A0EF8
:1015F000E66ED9DCE5520D0EE66ED5DCE552500EF6
:10160000E66ED1DCE552720EE66ECDDCE552650E7B
:10161000E66EC9DCE552730EE66EC5DCE552730E6C
:10162000E66EC1DCE552200EE66EBDDCE552220E10
:10163000E66EB9DCE552410EE66EB5DCE552220EEF
:10164000E66EB1DCE552200EE66EADDCE552660ECC
:10165000E66EA9DCE5526F0EE66EA5DCE552720E71
:10166000E66EA1DCE552200EE66E9DDCE552610ED1
:10167000E66E99DCE552750EE66E95DCE552640E79
:10168000E66E91DCE552690EE66E8DDCE5526F0E7A
:10169000E66E89DCE552200EE66E85DCE552740EBE
:1016A000E66E81DCE552650EE66E7DDCE552730E7A
:1016B000E66E79DCE552740EE66E75DCE552200EBE
:1016C000E66E71DCE5529EAAFED7410EAE5C07E1E4
:1016D0006FEC10F066EC11F05CEC11F0FFD722EC2F
:1016E00004F0E552E552E7CFD9FF1200040118518A
:1016F000600BE842E842E842E842E842000901E0C3
:1017000055D01951070A51E00B0A4FE0070A40E093
:10171000010A2CE00B0A28E0020A26E0030A22E074
:10172000080A12E0010A0EE00F0A0AE0030A01E0CB
:101730003CD00101010E0B6F0101040E126F36D077
:1017400036D834D090D832D00101010E0B6F010190
:10175000140E0C6F010E0D6F010113930101010EA8
:10176000106F24D0A8D822D0F6D820D00101010EC5
:101770000B6F04011C5101010C6F0D6B150E0C2732
:10178000010E0D23010113930101010E106F0ED004
:101790000101010E0B6F04011C51EA6A150FE96E7D
:1017A000010EEA221AC4EFFF01D000D01200800E11
:1017B0000401185D57E11B51030A34E0010A10E0EF
:1017C000030A01E04DD00101010E0B6F0101DE0E95
:1017D0000C6F220E0D6F120E0101106F116B40D0B5
:1017E0000101010E0B6F04011A51F66EF76AD890D1
:1017F000F636F7368C0EF626230EF7220900F5CFC3
:101800000CF10A00F5CF0DF1020E0101F76A0C256B
:10181000F66E0D51F7220900F5CF10F10A00F5CF51
:1018200011F11ED00101010E0B6F04011A51F66E69
:10183000F76AD890F636F736900EF626230EF72282
:101840000900F5CF0CF10A00F5CF0DF10CC1F6FF40
:101850000DC1F7FF0800F5500101106F116B00D0AA
:101860000101138312000101010E0B6F0F0EE66ED2
:10187000710EE66E0F0EE66ECBEC0FF0E552E55200
:10188000E552010EE66E150EE66E010EE66ECBEC2D
:101890000FF0E552E552E5521AC414F104011A5151
:1018A00004E10101050E126F05D00101060E126F51
:1018B000E0EC0FF012000401206B216B04011851C1
:1018C0001F0B020A16E0030A10E0010A01E035D0FE
:1018D0000101010E0B6F80A402D0040120810101DF
:1018E00013A102D00401208328D00101010E0B6F47
:1018F00024D00101010E0B6F04011C510F0B080DC8
:10190000F350116A000F106E040E11221C51800B4F
:1019100001E0010E040DF350010110240E6F000EC2
:1019200011200F6F0EC1E9FF0FC1EAFFEF50040B4A
:1019300003E00401010E206F00D001010B050AE154
:101940000101200E0C6F040E0D6F010113930101B4
:10195000020E106F120004011A0510E118511F0B3E
:1019600000090CE10101010E0B6F030E0401195D6A
:1019700003E10101138102D00101139104011A5105
:101980003AE118511F0B020836E11C510F0B0009F8
:1019900032E00101010E0B6F04011C510F0B080D09
:1019A000F350116A000F106E040E11221C51800BAF
:1019B00001E0010E040DF350010110240E6F000E22
:1019C00011200F6F030E0401195D07E1840E0EC193
:1019D000E9FF0FC1EAFFEF6E0ED01CAF06D00EC1BB
:1019E000E9FF0FC1EAFFEF6A06D0880E0EC1E9FFDA
:1019F0000FC1EAFFEF6E12006C5002E0000E01D042
:101A0000010E00090BE0040100513C0BE842E842E2
:101A10000D0802E10CD801D01CD808D06C5002E0AF
:101A2000000E01D0010E040901E023D81200D9CF25
:101A3000E6FFE1CFD9FFE65201010A6B0B6B106B99
:101A4000116B76EC0BF0DDD8E552E552E7CFD9FF0C
:101A50001200020E01010A5D0AE196D8040100BDE0
:101A600003D0C80E006F02D0880E006F01D00FD9CE
:101A70001200040E0101125D0AE11AC46EFF6E50DD
:101A8000000803E2050E126F02D0030E126F01016F
:101A90000A050AE10BD8040104BD03D0C80E046F87
:101AA00002D0880E046F01D0F2D81200D9CFE6FF21
:101AB000E1CFD9FF020EE1260101080E105D000EF4
:101AC000115905E210C1DEFF11C1DDFF03D0080E80
:101AD000DE6EDD6A040104930491010EDB500413F1
:101AE000DFCF05F4000EDB500101105F010EDB506B
:101AF000115B200E0E6F040E0F6F010113A31ED099
:101B0000D9CFE9FFDACFEAFFEE50ED1016E00CC1B5
:101B1000F6FF0DC1F7FF0800F5500EC1E9FF0FC138
:101B2000EAFFEF6E01010E2B000E0F230C2B0D238D
:101B3000DF06010E01E2DB06E3D71CD0D9CFE9FFB7
:101B4000DACFEAFFEE50ED1015E00CC1E9FF0DC150
:101B5000EAFFEF500EC1E9FF0FC1EAFFEF6E01018E
:101B60000E2B000E0F230C2B0D23DF06010E01E2BE
:101B7000DB06E4D7020EE15C02E2E16AE552E16EC7
:101B8000E552E7CFD9FF1200D9CFE6FFE1CFD9FF69
:101B9000020EE126030E04010015E76E010EE7CFE9
:101BA000DBFF01C4DFFFDE5001011027DD501123F0
:101BB000200E0C6F040E0D6FD9CFE9FFDACFEAFFCC
:101BC000EE50ED1014E00CC1E9FF0DC1EAFFEF503B
:101BD0000EC1E9FF0FC1EAFFEF6E0E2B000E0F23BF
:101BE0000C2B0D23DF06010E01E2DB06E5D7020E0A
:101BF000E15C02E2E16AE552E16EE552E7CFD9FF2E
:101C0000120001010B510CE10401080E016F180EC6
:101C1000026F040E036F840E006F0401046F35D051
:101C2000040118AF22D00101105104011E5D010111
:101C3000115104011F5904E21EC410F11FC411F117
:101C400035DF0101010E0A6F0401080E016F180E45
:101C5000026F040E036F800E006F0401200E066FEA
:101C6000040E076FC80E046F10D00101020E0A6F38
:101C70000401056BC80E046F0401080E016F200EED
:101C8000026F040E036FC80E006F6D981200010101
:101C90000A6B0401080E016F180E026F040E036F29
:101CA000880E006F0401046B12008A849394E66A24
:101CB000030EE66E020EE66E52EC12F0E552E552AD
:101CC000E5520001870EF36F0C0EF46F79EF0EF002
:101CD0008A94C2EC12F00001F46FC2EC12F0000121
:101CE000F36F8A84F3B502D0000E02D0010E00D04B
:101CF0001200D9CFE6FFE1CFD9FF030EE126F3C0F2
:101D000010F0F4C011F0D89011321032E804FBE169
:101D100010C0DEFF11C0DDFFD950010FE96EDACF30
:101D2000EAFFEF50100B08E1010EDB9ADB9CDB9E13
:101D300000012B0EF56F16D0010EDB8ADB8CDB8EDB
:101D400000012D0EF56FDECF10F0DDCF11F0FF0E8C
:101D5000101A111A10C0DEFF11C0DDFFDF2A010EBC
:101D600001E3DB2ADECF10F0DDCF11F00A0E110205
:101D7000F3CF11F01002F3CF10F0F4501126040E3F
:101D8000D89011321032E804FBE110C0DEFF11C020
:101D9000DDFF040EF36E020EF3CFDBFFDB50000815
:101DA00033E2DECF10F0DDCF11F00A0E0B6E0C6ABD
:101DB00010C006F011C007F0A0EC12F002C010F045
:101DC00003C011F00F0E10143009E66E020EDB5046
:101DD000EA6AF50FE96E000EEA22E552E750EF6E6F
:101DE000D9CFE9FFDACFEAFF0A0E0B6E0C6AEECF0D
:101DF00006F0EDCF07F0A0EC12F006C0EEFF07C032
:101E0000EDFF020EDB06CAD7300E0001F65D07E1DA
:101E1000200EF66F300EF75D02E1200EF76FF9C06D
:101E2000FAF02E0EF96FF80EFB6F430EFC6F0D0EDD
:101E3000FD6FFE6B030EE15C02E2E16AE552E16ECA
:101E4000E552E7CFD9FF120080A203D06DA60FD8CC
:101E500002D06DB613D80101120508E16DBA06D0A3
:101E6000686A696A69806988020E126F12006D6A79
:101E7000696A6D860101010E126F12006D6A696A4E
:101E80000101126B12003EEF0FF00101125101E14E
:101E90003AD06850040B04E06950040B01E038D8D4
:101EA0006DB231D06850010B04E06950010B01E0C4
:101EB00050D86850100B04E06950100B01E024D892
:101EC0006850400B04E06950400B01E037D868507F
:101ED000200B04E06950200B01E032D86850020B5F
:101EE00004E06950020B01E032D8030E0101125DDB
:101EF00001E209D06850080B06E06950080B03E0C6
:101F0000FCEC0CF068961200698468986D821200EF
:101F10006D92699468941200010113A10ED0F8DF4C
:101F20006D840101080E166F070E176F1607000E5D
:101F3000175B16511711FAE16D941200689C12009C
:101F400070A003D047EC0EF07090689A120068926F
:101F500012006A6A686A9F0E6B6E7B0E696E6E6A0B
:101F60000F0EE66E710EE66E0F0EE66E14D8E55299
:101F7000E552E552160E706E68A602D06896FCD740
:101F80006D9847EC0EF0010113910101146B0101F2
:101F9000030E126F1200D9CFE6FFE1CFD9FFFD0E7D
:101FA000DBCFE9FFFE0EDBCFEAFFFC0EDB5004E0E7
:101FB000EE6AFC0EDB06F9D7E552E7CFD9FF120037
:101FC0000001FF6B1E0E716E0401400E096F280E9A
:101FD0000A6F040E0B6F880E086F0401680E0E6FF7
:101FE000040E0F6F400E0C6F1200D9CFE6FFE1CF49
:101FF000D9FFE652FC0EDB50400805E2400EF36EBE
:10200000FC0EF3CFDBFFDF6AFC0EDB50DF5C19E276
:10201000DF50E76EFD0EDBCFE9FFFE0EDBCFEAFF00
:10202000E750E926000EEA22EF50E66EDF50EA6A3A
:10203000680FE96E040EEA22E552E750EF6EDF2AE0
:10204000E3D7FC0EDBCF0DF4400E04010C170C7D22
:10205000880E0C13E552E552E7CFD9FF1200D9CF15
:10206000E6FFE1CFD9FF0001FF6B040108BF30D0CC
:10207000FC0EDBCF10F00951D880105403E2FC0EA7
:1020800009C4DBFF0001FF6BFC0EDB50FF5D19E2B2
:10209000FF51EA6A280FE96E040EEA22EF50E66E5D
:1020A000FF51E76EFD0EDBCFE9FFFE0EDBCFEAFF4F
:1020B000E750E926000EEA22E552E750EF6EFF2BCB
:1020C000E3D70401400E096F0817087D880E081336
:1020D0000001FF5100D0E552E7CFD9FF1200C26ADC
:1020E000C16ABC0EC06E92681200D9CFE6FFE1CF84
:1020F000D9FF020EE126DE6ADD6A110EC26EC282CF
:10210000C2B2FED7C3CFDEFFC4CFDDFF010EC26E69
:10211000DECF10F0DDCF11F010C0F3FF11C0F4FFDF
:10212000020EE15C03E200D0E16AE552E16EE552A5
:10213000E7CFD9FF1200D9CFE6FFE1CFD9FF080ED4
:10214000E126DE6ADD6A020EDB6A030EDB6A040E3C
:10215000DB6A050EDB6A060EDB6A070EDB6ADE6AE7
:10216000DD6ADECF10F0DDCF11F0010E105C000E45
:10217000115819E2BADFF3CF10F0F4CF11F0126A60
:10218000136AD950040FE96EDACFEAFF1050EE2639
:102190001150EE221250EE221350EE22DF2A010ED1
:1021A00001E3DB2ADED7040EDBCF06F0050EDBCF22
:1021B00007F0020E06C0DBFF030E07C0DBFF020EB6
:1021C000DBCF10F0030EDBCF11F0D89011321032BC
:1021D000D8901132103210C0F3FF11C0F4FF080E76
:1021E000E15C03E200D0E16AE552E16EE552E7CF3F
:1021F000D9FF1200D8CFE4FFE0CFE4FFE46EDACFDE
:10220000E4FFE2CFDAFFE9CFE4FFEACFE4FFF6CF65
:10221000E4FFF7CFE4FFF5CFE4FFF3CFE4FFF4CF23
:10222000E4FFFACFE4FF00EE00F0100EE80403E351
:10223000EECFE4FFFBD700EE10F0040EE80403E35A
:10224000EECFE4FFFBD7E6529E50010B0CE09D5011
:10225000010B09E0CD90CE6ACF68CD809E909BECBB
:1022600010F0F350BB6EE55200EE13F0040EE804DC
:1022700003E3E5CFEDFFFBD700EE0FF0100EE8040F
:1022800003E3E5CFEDFFFBD7E5CFFAFFE5CFF4FFA2
:10229000E5CFF3FFE5CFF5FFE5CFF7FFE5CFF6FF9D
:1022A000E5CFEAFFE5CFE9FFE5CFDAFFE550E5CF7F
:1022B000E0FFE5CFD8FF1000010ECD6E9E909D800F
:1022C000CE6ACF689F90F28EF28C12009482CB6817
:1022D000BB6AFC0EBA6E040ECA6E94921200120112
:1022E000000200000008D8040C00000001020001F8
:1022F00009022000010100803209040000020000F0
:10230000000007050103400020070581034000206D
:102310000403090434034D006900630072006F0078
:1023200063006800690070002000540065006300CD
:1023300068006E006F006C006F006700790020007D
:1023400049006E0063002E00440350004900430022
:10235000440045004D002000460053002000550079
:10236000530042002000440065006D006F00200013
:1023700042006F00610072006400200028004300EA
:10238000290020003200300030003400F022F0221A
:102390001023142348232A0EF66E080EF76E000E43
:1023A000F86E01010900F550056F0900F550066F40
:1023B00003E1056701D03DD00900F550006F090029
:1023C000F550016F0900F550026F09000900F55042
:1023D000E96E0900F550EA6E090009000900F550A0
:1023E000036F0900F550046F09000900F6CF07F1EB
:1023F000F7CF08F1F8CF09F100C1F6FF01C1F7FFEF
:1024000002C1F8FF0101035302E1045307E0090090
:10241000F550EE6E0307F8E20407F9D707C1F6FF9F
:1024200008C1F7FF09C1F8FF01010507000E065BAF
:10243000BFD7120004500902F3CF00F0F4CF01F02F
:102440000A02F3500126000EF420026E04500B0223
:10245000F3500226000EF420036E04500C02F350D9
:10246000032605500902F3500126F4500222000E03
:10247000032205500A02F3500226F45003220550AD
:102480000B02F350032606500902F3500226F450C3
:10249000032206500A02F350032607500902F350A4
:1024A00003261200D9CFE6FFDACFE6FFE1CFD9FF4E
:1024B000E2CFDAFF3F0EC716C66AFD0EDB50C6122A
:1024C000FB0EDB50C712FC0EDB50030A09E0010AC9
:1024D00004E0020A06E1C78C04D0C78CC68801D08C
:1024E000C688FD0EDB50050A03E0010A04E1928A6A
:1024F0009382C79E01D09392949E9380C68AE552A0
:10250000E5CFDAFFE7CFD9FF120005D812D81CECCF
:1025100006F0FCD712000F0EC11292829284140EA4
:102520006F6E0101126B0101136B0101146B22EF3D
:1025300004F024EC0FF06FBE02D045EC0FF0120057
:10254000036A026A100EE76ED89006360736023626
:1025500003360B50025C0C50035805E30B50025E2F
:102560000C50035A062AE72EF0D7120013EE00F0A3
:1025700023EE00F0F86A0F9CCBEC11F085EC12F022
:10258000FDD71200C96AC7A0FED7C95012000000CB
:1025900005F00700000000000000000000FFFFFF42
:0200000400F00A
:10000000FFFFFFFFFFFFFFFFFFFFFFFFFFFFFFFF00
:10001000FFFFFFFFFFFFFFFFFFFFFFFFFFFFFFFFF0
:10002000FFFFFFFFFFFFFFFFFFFFFFFFFFFFFFFFE0
:10003000FFFFFFFFFFFFFFFFFFFFFFFFFFFFFFFFD0
:10004000FFFFFFFFFFFFFFFFFFFFFFFFFFFFFFFFC0
:10005000FFFFFFFFFFFFFFFFFFFFFFFFFFFFFFFFB0
:10006000FFFFFFFFFFFFFFFFFFFFFFFFFFFFFFFFA0
:10007000FFFFFFFFFFFFFFFFFFFFFFFFFFFFFFFF90
:10008000FFFFFFFFFFFFFFFFFFFFFFFFFFFFFFFF80
:10009000FFFFFFFFFFFFFFFFFFFFFFFFFFFFFFFF70
:1000A000FFFFFFFFFFFFFFFFFFFFFFFFFFFFFFFF60
:1000B000FFFFFFFFFFFFFFFFFFFFFFFFFFFFFFFF50
:1000C000FFFFFFFFFFFFFFFFFFFFFFFFFFFFFFFF40
:1000D000FFFFFFFFFFFFFFFFFFFFFFFFFFFFFFFF30
:1000E000FFFFFFFFFFFFFFFFFFFFFFFFFFFFFFFF20
:1000F000FFFFFFFFFFFFFFFFFFFFFFFFFFFFFFFF10
:020000040030CA
:0E000000240E3F1E008181000FC00FA00F4094
:020000040020DA
:08000000FFFFFFFFFFFFFFFF00
:00000001FF
